:020000040000FA
:060000000219FD0200C818
:03000B0002008D63
:03002B000200923E
:03005B000202C5D9
:030073000200B5D3
:100080000406080C10182030406080A0C0C28D0506
:100090004032C0D0C0E0C2CF0541E5646009E563ED
:1000A000600575630001B0756301E52360021523E7
:1000B000D0E0D0D032C2AF53E67F7592FA7593FF8D
:1000C000C22053917FD2AF32C0D0C0E0C0F0D2D3B3
:1000D0005388EFA88AA98CAA40308D010A758A003E
:1000E000758C00754000438810E564700AC3E833DE
:1000F000F8E933F9EA33FA30331FE8C4540FFAE968
:10010000C454F04AFAC3132AFAC3E833F8E933F9BE
:10011000E82AFAE93406FB216C30320FC3E833E9F0
:1001200033FAE82AFAE93400FB216C303115E8751E
:10013000F056A4AAF0E975F056A42AFAC5F03400E6
:10014000FB216CC3EA13FAE913F9E813F8E875F038
:1001500056A4AAF0E975F056A42AFAC5F03400C3F3
:1001600013FBEA13FAC3EB13FBEA13FAC3EB941283
:100170005006C3EB9406501A0522E52270021522A0
:10018000C3E522940A500241BB7552007A007B00FD
:10019000418DE522600215223035067C007D082164
:1001A000ACAC31AD32303A04AC33AD34C3EA9CFA76
:1001B000EB9DFB9208AE5EAF5F303A4250072034B1
:1001C00009D23421CA303402C234303404AE60AFB4
:1001D00061203902B234C3EA33FAEB33FBA2085090
:1001E0000AEAF42401FAEBF43400FBC3EA9450FA6F
:1001F000EB9400FB501478007A007B00410AA208BF
:10020000500878007A007B004169E5255403601BA3
:10021000202A18E55B33F9EB7007C3E99A4002E93D
:10022000FAE53CC4332AFAEB3400FBEA8EF0A4F979
:10023000AAF0EB8EF0A42AFAC5F03400FBC3EB134E
:10024000FDEA13F8C3ED13FDE813F80FEF14600493
:10025000C3E833F8C3E933EA33FAEB33FBDFEDEB02
:1002600030E30678FF7AFF7B078852D230C3E894E8
:10027000404002D221C3E559FC955A4003AC5AC311
:10028000EC95525008EC75F008A4FAABF0EAF4F8DB
:10029000EBF45407F98854895575230AE55830E280
:1002A0000DD0F0D0E0D0D053F7DF43F74032D0F09C
:1002B000D0E0D0D053D8FE43DA013275230AD0F013
:1002C000D0E0D0D032C0D0C0E0D2D38554FB855529
:1002D000FC85555853F7BF53DAFEC3E552940140ED
:1002E0000575530041F1E5532401F553500375534F
:1002F000FF53F7DF53D8FED0E0D0D032790180141D
:1003000079038010790A800C791E80087964800452
:1003100079C880007817E4D5E0FDD8FAD9F6227ABA
:10032000147B7880127A107B8C800C7A0D7BB480E1
:10033000067A0B7BC880007902E4C293D5E0FDD237
:1003400092D293D5E0FDC293D5E0FDC292D293D56F
:10035000E0FDE920E004D290D29130E004D294D2C2
:1003600095E562D5E0FDE920E002C29130E002C2ED
:10037000957496D5E0FDD9C1EAF8D5E0FDD8FBDB50
:10038000B6C2932278FFC22120283D202912D22113
:10039000C3E548940A4009C3E55294405002C22183
:1003A00079A1E76023E548601F74FF8548F08485E4
:1003B0003FF030290375F005A4F8C5F0600278FF1E
:1003C000C3E8955B5002A85B885A22C3E54794A016
:1003D000E5489400E55A50031461DC046002F55AC4
:1003E0002275E89022055CC3E55C94084055E5E879
:1003F00020ECF2A8BDA9BE755C00E9FA79A0E7601F
:1004000041EA7006E55D6018800CC3E8955D600EFA
:10041000E55D5005600A1480070460FA8002E55D1E
:10042000F55DC394F6401B7559C0C394064013751F
:100430005980C39406400B755940C3940640037518
:10044000590022E5592410500274FFF559227432E4
:1004500079A687F0A4C5F0A2F733F8C3E895594010
:1004600002A859885B227547007548F022C2AF7513
:10047000C800A8CCA9CDAA4130CF010A75C804D2C2
:10048000AFC3EA13FAE913F9E813F8AB42AC4388B7
:10049000428943C3E89BF8E99C20280A547FF9303D
:1004A0002C02A18781E4AD448A44F9EA9D547FFA85
:1004B000600478FF79FFAE45AF468B458C46A84275
:1004C000A943C3E89EF8E99FF9C3E54813FBE54754
:1004D00013FAE82AF547E93BF54850067547FF75DA
:1004E00048FFA12EAA47AB48AC47AD487E047F0227
:1004F000C3EB9404400A1E1FC3EB940840021E1F66
:10050000C3ED13FDEC13FCDEF7C3EA9CFAEB9DFB95
:10051000EF6009C3E913F9E813F8DFF7EA28FAEB0B
:1005200039FB8A478B4850067BFF8B478B48C3EBD0
:1005300094025002D22C3028047F03A1597892E60D
:10054000FFC3E53D948240110FC3E53D94A04001F7
:100550000FC3EF940640027F057E02E548C4540FA6
:10056000F9E548C454F0F8E547C4540F28F8C3E847
:100570009EFAE99400FB4009C3EA9401EB94005011
:10058000047A01E4FBA1D3AA47AB48EBC4FEEAC45A
:10059000540F4EFCC3EA9CFAEB9400FBC3E813C370
:1005A00013F8EA28FAEB3400FB8A478B48C3EB9434
:1005B000024002C22C7802EBC4FE7B00EAC4540F56
:1005C0004EFAC3EA98FA4005C3940150027A0178C2
:1005D00092E6FF30200280FB854E92854F93D22019
:1005E00043E680C3E49AF8E49BF9C3E833F8E933BF
:1005F000F9302C02C165E8FAE9FBD3E913FDE813F1
:10060000FC884E894FC3EF94036037EF20E00CE87D
:100610002CF8E93DF9ECFAEDFB8013E828F8E9390C
:10062000F9C3E82401F8E93400F97AFF7BFFC3EF4E
:100630009403400E8A508B51884A894B8C4C8D4DC7
:10064000C199885089518A4A8B4B8C4C8D4D3028EA
:10065000127550F07551FF754CF0754DFF754EF0E9
:10066000754FFFC199E8FAD3E813FC884EC3EF94A5
:10067000036020EF20E007E82CF8ECFAC185E828B9
:100680002401F87AFFC3EF940340088A50884A8C0B
:100690004CC19988508A4A8C4C302002C199753AD5
:1006A00002D22043E680E5255403602DA847A948DF
:1006B000C3E913F9E813F8302804E92440F9C2AF7C
:1006C00053E67F759100C3E498F594E499F5957528
:1006D0009104D22043E680D2AF22D2227549007520
:1006E0002000302B03752040800ED2227549007502
:1006F0002040302B0375200078017901202C20E563
:100700002554036002C2227914E548C31370010422
:10071000F8C3941440027814302804781B791BC362
:10072000E833F8C3E933F9202010E549600C30289C
:1007300003D53A04D224E1AFD1A10549E59B544049
:10074000B52002E19930280908C3E899400118E171
:100750002720220A08C3E8994002C1F8E127C222F3
:10076000C2AF53E67F759100302C127594007595D9
:10077000FC759104D22043E680D2AFC1F8AE47AFFA
:1007800048C3EE33FEEF33FF50047EFF7FFFC3E428
:100790009EF594E49FF595E171C3E539940150020B
:1007A000C1F8302202C1F8D802E1ADE127C224C26B
:1007B000AF53E67F759100855094855195759104EE
:1007C000854A92854B93D22043E680D2AFE52554EB
:1007D0000360072029020539801030240D202B0AE0
:1007E00020220715811581020F3A22780030210559
:1007F0003022027801E53D75F007A4F9E5F028F50F
:10080000F0E9A2F013A2F113A2F213F53DC394781C
:100810005003753D78C3E53D953E400BD223C29110
:10082000C293C29575D57F30200280FB854C92859E
:100830004D93D22043E68022203814C2AFC293C227
:1008400090D291D29575D56FD2AF759F20213CC2C1
:10085000AFC293C294D295D29175D57ED2AF759F17
:1008600020213C203815C2AFC295D29375D57BC2EA
:1008700090D291D2AF759F3002093CC2AFC291D2E3
:100880009375D57BC294D295D2AF759F1002093C67
:10089000203814C2AFC291C294D295D29375D57B41
:1008A000D2AF759F10213CC2AFC295C290D291D2F7
:1008B0009375D57BD2AF759F30213C203815C2AFE0
:1008C000C293D29175D57EC294D295D2AF759F2036
:1008D00002093CC2AFC293D29575D56FC290D29136
:1008E000D2AF759F2002093C203814C2AFC295C216
:1008F00092D293D29175D57ED2AF759F30803DC292
:10090000AFC291C292D293D29575D56FD2AF759F77
:10091000108029203814C2AFC291D29575D56FC20C
:1009200092D293D2AF759F108012C2AFC295D2916E
:1009300075D57EC292D293D2AF759F30C22322C2A8
:1009400091C293C295C291C293C29575D57F227808
:100950008076FF0876FF0876FF0876FF0876FF08A6
:1009600076FF0876090876FF087601788C7601080C
:1009700076FF0876FF0876FF0876FF0876FF087690
:10098000030876FF0876FF0876FF0876250876D0FC
:100990000876280876500876040876FF087602085C
:1009A00076FF08767A0876FF0876010876010876E1
:1009B000FF0876FF08760008760022FA75F00CA48E
:1009C000ABF0EAC333F8740133F9E8C333F8E93321
:1009D000F9E8C32BF8E93400F9E8C333F8E933F94F
:1009E000227888E6C39403D23A5002C23AC238E66B
:1009F00030E102D238A23892397886E6149000802D
:100A00009378A6F67886E6F53FC394025003753FC7
:100A100002789CE6753EFFB40203753EA0B4030362
:100A2000753E827896E631BB88318932789EE63110
:100A3000BB883389347897E631BB88358936313FB6
:100A4000223035117A007B007CFF7D007E0051A8AA
:100A50008B5F8A5E22303A227896E6FA7B00789E97
:100A6000E6FC7D00C3EA33FAEB33FBC3EC33FCED69
:100A700033FD7E0A51A88B618A607896303A0278FD
:100A80009EE6FA7B007897E6FC7D007E00303A1007
:100A9000C3EA33FAEB33FBC3EC33FCED33FD7E0AE0
:100AA00051A88B5F8A5E2222C3EC9EFCED9400FD70
:100AB000C3EC9AFCED9BFDC3EC9423ED9400500431
:100AC0007C237D00C3EC94FFED940140047CFF7D0A
:100AD000017BFF0B7A000AEA7009C3EC33FCED33AB
:100AE000FD41D3EC8AF0A4AEF0ED8AF0A42E947C04
:100AF00040E4EAF460DD22D23551411203087A0065
:100B00007B007C10120300E5522AFA74003BFBDCE8
:100B1000F37C04C3EB13FBEA13FADCF7FFEB600290
:100B20007FFFC23551412278A5E6F95403D2867081
:100B300002C286E9540CD2877002C287E95430D2CF
:100B4000967002C296E954C0700022E5EF20E603D9
:100B50007520000520903FFFE520146006901DFFE2
:100B60001460009304600375EF127597DE7597ADFE
:100B70007581C043FF801202FC75EF0275A9003138
:100B80003F75803F75F1F075A4C075803F75D4FF47
:100B900075900075F27F75A57F75900075D57F758E
:100BA000A60175E34075E202C291C293C295120399
:100BB0000CC290D291C292D293C294D2951202FCEE
:100BC000C291C293C295313FE4F8F6D8FD314FF19E
:100BD0008178988662753001C2AF12031012031F2C
:100BE00012030812032512030812032B12030871C3
:100BF00027C2AF78FA79FA308507D9FBD8F7021CFB
:100C00000031E1514178988662313F75A91375A78B
:100C10001075C10075A70075640075E4057588112D
:100C2000758E0475890975C80475910475D8407569
:100C3000D90875F783759E0075960275DA4A75DBDB
:100C40000075A82375E69075F310759B80759D005F
:100C500075D12C75BCC075BB1075E88075B20112DA
:100C600002FCD2AF753C00C230120310C2317522B3
:100C70000012030CC3E522940A4024D231C232751B
:100C8000220012030CC3E522940A4013D232C2336D
:100C900075220012030CC3E522940A4002D23312DB
:100CA0000300203003020BF1C2AF12031F12031F17
:100CB00012031FD2AF120310303A02A14B120300ED
:100CC000788CE6C394015002A14BE530C3940150E7
:100CD00002A14B7F02D235514112030CC2AFC23583
:100CE0005141AE52C3E552947FD2AF405E1202FC36
:100CF000C2AF120331D2AFDFDC51F7C3EF7897F602
:100D0000120310F1BF12106A7F0AD235514112034B
:100D10000CC2AFC2355141AE52C3E552947FD2AF3F
:100D200050E61202FCC2AF12031F12030412031F8B
:100D3000D2AFDFD651F7EF24037896F6120310F105
:100D4000BF12109912030C514161F112030C78018A
:100D5000303A027805C3E55298400281B8C2AF121A
:100D60000331120331120331D2AF12031075300078
:100D7000E4F537F5380537E537F4703E0538789AED
:100D8000E67819146012783214600D787D146008CA
:100D900078FA146003753800C3E53898401C313F79
:100DA0001202FC153875370078998662C2AF1203BB
:100DB00031D2AF7898866212030C120304E52370D7
:100DC0000261F17801C3E5529840AA12030CE523B1
:100DD0007003020BF1C2AF313FE4D2AFE4F55CF532
:100DE00024F525F53D755C081202FC1203E1E5E8E7
:100DF00020ECFBA8BDA9BEE97001F8885D1203E5EF
:100E0000755C08C2AF7559FF12044E855B59855B4E
:100E10005AD2AF75A71075C13075A70075A90375B3
:100E20006401303A07C238303402D238D2287539DA
:100E30000011E8311312046612046D1204661204E4
:100E40006D1204661206EA1207EB113812046D12D5
:100E500006DA202C03120384302C031203CB120772
:100E6000EB116312046D1206EA1207EB11901204E3
:100E70006D1206DA1207EB11BB12046D1206EA12AC
:100E800007EB11E812046D1203E11206DA1207EB08
:100E900031131203E512046D302827855B59791848
:100EA0007A0CC3E53999400EC228D2298A3B855B6A
:100EB00059855B5A800CC3E55294014003020E44ED
:100EC000E14230291C202B19E53B147006C229D2BF
:100ED0002AC144F53BC3E55294014003020E44800D
:100EE00061753C0078FA79A4E760027803C3E553A2
:100EF00098504FE523604B303A17203805203407CF
:100F0000800F303402800A202B07D22B855B59C119
:100F10007178F0302B05855B597820C3E5489850EF
:100F200003020E44302B1BC22BC238303402D2389D
:100F3000D229753B12855B59C144053CE5526002DC
:100F4000E145753C00C2AF313F7524007525007541
:100F5000A91375A71075C10075A700756400D2AFFD
:100F600012030C313F78A4E6600CC290D291C29279
:100F7000D293C294D295C3E53C9404400261F1A19E
:100F800070901A0D7820121001E520B4550BA312B1
:100F90001001E520B4AA028006314FF1BF801F90F6
:100FA0001A0378807B0A121001A308DBF9901A0F4C
:100FB000788C7B1A121001A308DBF9901A2922C23F
:100FC000AF12104012101A901A007410121006A3DB
:100FD0007401121006A37420121006901A03788070
:100FE0007B0A121005A308DBF9901A0F788C7B1A84
:100FF000121005A308DBF9121053121031901A29B0
:1010000022E493F622E6438F01538FFD75EF0275BC
:10101000B7A575B7F1F0538FFE22438F02438F01BE
:1010200075EF0275B7A575B7F1901A0DF0538FFCE7
:1010300022901A0D74551106901A0E74AA110622E8
:101040007A3079D07820901A401101E520F709A371
:10105000DAF7227A3079D0901A40E7110609A3DA3C
:10106000F9227C05120310DCFB22C2AF12031F120F
:10107000032512032B12033112030412031F120360
:101080002512032B12033112030412031F1203252E
:1010900012032B120331D2AF22C2AF12033112035B
:1010A0002B12032512031F12030412033112032B08
:1010B00012032512031F12030412033112032B1211
:0810C000032512031FD2AF2229
:1019FD00020B4B100120FFFFFFFFFFFF09FF01FF4F
:101A0D0055AA01FFFFFFFFFF03FFFFFF25D0285061
:0D1A1D0004FF02FF7AFF0101FFFF0000FF40
:101A400023455F485F3030232020202020202020A5
:101A500023424C48454C492445464D3842323123B7
:101A60002020202020202020202020202020202076
:101C0000C2AFC2D37597DE7597AD7581C075A90057
:101C100043FF80752438752503B1C875EF0243F181
:101C20002053A4DFD28575D4FF75E3407DFA780395
:101C300079E67C10752200752300901DD57B067512
:101C400024987525013085028145208508D8FBD967
:101C5000F9DCF781B7308508D8FBD9F9DCF781B713
:101C6000B188E493A3C39A6004DDC381B7DBDBB121
:101C70007A6002812E7B08E493FAA3B15BDBF87AE9
:101C800030B15B752200752300B17AEAFCEBFDC32D
:101C9000ED94FE400EB17A8A278B28ED30E0048A5D
:101CA000828B83B17A7AC270D8C3ED94FE601350F0
:101CB000CEBD0023EC60097520007521FF020000F5
:101CC0008100A827A9280809D804D90281D4B17EA7
:101CD000EAF281C80D81A3C3ED94035047EDA2E061
:101CE00092007AC5C3E5829400E583941C5092204B
:101CF0000010438F02438F0175B7A575B7F1F0301F
:101D0000001DA827A9280809438F01538FFDD80477
:101D1000D902A11FE275B7A575B7F1F0A3A10E53C3
:101D20008FFC817F7AC1BD030CE493A3FAB13FDC41
:101D3000F8B137817F8181AA22AB23B15BEBFAEA4C
:101D40006222752608C3E52313F523E52213F52245
:101D500050066323A0632201D526EAB1C8B1C87535
:101D6000260AEAF4200102D285300102C285B1C8F8
:101D7000C3134002C201D526EB22B17EEAFB2085C7
:101D800002A17E308502A183752608AE24AF25C34B
:101D9000EF13FFEE13FEB1CCB1C8C3EA13308502D6
:101DA0004480FA30E703632201C3E52313F523E5FA
:101DB0002213F52250066323A0632201D526D9E51C
:101DC0002265236523F52222AE24AF250E0FDEFE09
:101DD000DFFCD20122424C48656C6934373163E83C
:031DE000B2060147
:00000001FF
